:08000000803102288731E52F51
:1005BC00640080010131890BDF2A00340D30833156
:1005CC004C2382310A3083314C2382310800012BB9
:1005DC007208840073088500000883314C23823133
:1005EC000130F2070030F33D0330F4009830890BF2
:1005FC00FD2AF40BFD2A7208840073088500120092
:10060C00031D092B0A2BEE2A08001F2B72088600EB
:10061C0073088700010883314C2383310130F207C2
:10062C000030F33D0330F4009830890B1B2BF40B96
:10063C001B2B72088600730887000108031D272BEB
:10064C00282B0C2B08002000B200AE1F2E2B2F2BBA
:10065C003F2B2D30B1003208860087013108810014
:10066C000130B1003108B207AD09AE09AD0A03196A
:10067C00AE0A2E08A5002D08A4003008A7002F08EC
:10068C00A60032088331E12383310800F10071099F
:10069C00F00070082000A0000830A1008C12632329
:1006AC00A00C03185B2B8C165C2B8C126323A10BF8
:1006BC00562B8C16632363236F2B1C30A200000077
:1006CC00000000000000A20B652B000000000000E1
:1006DC00080000000800780879040319762B772BA2
:1006EC00A02BFD01FD0A832B0130F835F90D890B88
:1006FC007B2B0130FC007C08FD07F91F862B872B18
:10070C007A2B79087B02031D8D2B78087A02031C47
:10071C00902B912B952B7808FA027908FB3B013032
:10072C00F936F80C890B962B0130FD02031D9F2B1B
:10073C00A02B872B7B08F9007A08F8000800F5013C
:10074C00F601700871040319AC2BAD2BDC2BF701EF
:10075C00F70AB92B0130F035F10D890BB12B0130B3
:10076C00F4007408F707F11FBC2BBD2BB02B013024
:10077C00F535F60D890BBE2B71087302031DC82BC2
:10078C0070087202031CCB2BCC2BD12B7008F202FD
:10079C007108F33B75140130F136F00C890BD22B38
:1007AC000130F702031DDB2BDC2BBD2B7608F1008F
:1007BC007508F00008002000AC002508AA002408E9
:1007CC00A9002708F1002608F0002A08F3002908E0
:1007DC00F2008331A523833171082000AA00700830
:1007EC00A9000130A8002808AC0729082A04031D19
:1007FC00002C012CE72B2C0886008701810101308D
:10080C00AC022708F9002608F8002508FB0024088C
:10081C00FA0083317123833178082000A80028085E
:10082C00AB002708F1002608F0002508F300240887
:10083C00F2008331A523833171082000A5007008D4
:10084C00A4000A302B02031C2C2C2D2C312C07302D
:10085C00A8002808AB073030A8002808AB072B08E5
:10086C00A8002C0886008701280881000130AC0202
:10087C0024082504031D432C442C072C0130A8000C
:10088C002808AC0708002000B900B101B2012630DD
:10089C00AC002C08B400562D25303A060319572C01
:1008AC00582C692C3A08AC003908860001308700B6
:1008BC002C0881000130AC002C08B9070130B107BD
:1008CC000030B23D562DB001A32C340886008701B0
:1008DC00403FB500413FB6000230AC002C08B407D5
:1008EC0035083604031D7B2C7C2C992CC430B500A8
:1008FC008930B600992C350884003608850000082C
:10090C00AC0039088600013087002C0881000130CA
:10091C00B5070030B63D0130AC002C08B9070130EA
:10092C00B1070030B23D350884003608850012004E
:10093C00031DA12CA22C812C562D2508AD002408BA
:10094C00AC00A40A0319A50A2C0884002D08850004
:10095C000008BA00003A03196A2D643A0319BD2C39
:10096C000D3A0319BD2C1A3A03196B2C562D340869
:10097C0086008701403FB700413FB8000230AC0011
:10098C002C08B407B81FCB2CCC2CD52C0330AC00C6
:10099C002C08B004B709B809B70A0319B80ABA0188
:1009AC00BA0A3A08AC00AD01AC35AD0D00302C07DD
:1009BC00840088302D3D8500003FAE00013FAF0024
:1009CC002F083802031DEC2C2E0837020318EF2CCD
:1009DC00F02CF12CFB2C0130AC002C08BA070530A4
:1009EC003A06031DFA2CFB2CD72C300803390319BB
:1009FC00002D012D112D2D30AC0039088600013051
:100A0C0087002C0881000130AC002C08B90701309C
:100A1C00B1070030B23D3A08AC002C08B3004D2DA4
:100A2C000A30F8000030F9003308AC00AD01AC35E9
:100A3C00AD0D00302C07840088302D3D8500003F23
:100A4C00F000013FF1003808F3003708F200833161
:100A5C00A52384317108FB007008FA0083317123DF
:100A6C0084317808303E2000AE002E08BA003A08D7
:100A7C00AC0039088600013087002C088100013059
:100A8C00AC002C08B9070130B1070030B23DFF3083
:100A9C00AC002C08B307330A031D552D562D162D0B
:100AAC002508AD002408AC00A40A0319A50A2C08DB
:100ABC0084002D0885000008AE002E08BA003A0804
:100ACC00031D692D6A2D522C3908860001308700D0
:100ADC0081013208A5003108A4000800F030210083
:100AEC00990098012200960121001A1F7E2D7F2D5E
:100AFC007A2D033022008C001F3021008C00230043
:100B0C008C01053024008C002100951322009D01DE
:100B1C0029302000BC009630BB007F30890B942D0F
:100B2C00BB0B942DBC0B942D2000A001A101A201A4
:100B3C00A301C101C2014108203E8600013087009B
:100B4C0081010130C1070030C23D003042024F30FC
:100B5C0003194102031CB32DB42DA12DC101C201F7
:100B6C004108A03E8600870181010130C107003099
:100B7C00C23D003042022F3003194102031CC72D25
:100B8C00C82DB62D8231E422853105302000BC0001
:100B9C000F30BB00F130890BD12DBB0BD12DBC0B11
:100BAC00D12D8231E42285318231E42285310A3023
:100BBC00F2008830F3008231ED2285314D30F200A5
:100BCC008930F3008231ED228531DA30F200883041
:100BDC00F3008231ED22853177302000A40088307B
:100BEC00A500A330A6008930A700BB30A80089302F
:100BFC00A9003830AA000930AB00203084314924D8
:100C0C00853120002508BE002408BD002030F200EC
:100C1C000130F30083310B2385314230F2008830F0
:100C2C00F3008231ED2285312E30F2008930F30051
:100C3C008231ED2285318231E42285310530F2009A
:100C4C008930F3008231ED2285317C30F20089301D
:100C5C00F3008231ED228531210015082000BB0004
:100C6C003B08C400AB30F2008830F3008231ED2237
:100C7C00853120004408BB00BC013B08AD003C089A
:100C8C00AE001030AF000030B000A030833129230B
:100C9C008531A030F2000030F30083310B23853115
:100CAC008231E4228531AF30F2008930F300823199
:100CBC00ED22853124000C082000BB003B08C40049
:100CCC004408BB00BC013B08AD003C08AE00103032
:100CDC00AF000030B000A030833129238531A03023
:100CEC00F2000030F30083310B2385318231E42292
:100CFC0085318231E42285312000C101C201FD2EF3
:100D0C009130F2008930F3008231ED2285312000E0
:100D1C000C08BB003B08C4004408BB00BC013B08EA
:100D2C00AD003C08AE001030AF000030B000A03079
:100D3C00833129238531A030F2000030F300833158
:100D4C000B238531093083314C2385312930200028
:100D5C00BC009630BB007F30890BB22EBB0BB22E81
:100D6C00BC0BB22E20000C1CBC2EBD2EC22E313062
:100D7C0083314C238531C62E303083314C23853161
:100D8C0020008C1CCA2ECB2ED02E313083314C231C
:100D9C008531D42E303083314C23853120000C1D0D
:100DAC00D82ED92EDE2E313083314C238531E22ED4
:100DBC00303083314C23853120000C1EE62EE72E7B
:100DCC00EC2E313083314C238531F02E3030833191
:100DDC004C2385310D3083314C2385310A308331DE
:100DEC004C23853101302000C1070030C23D00305A
:100DFC0042020A3003194102031C052F062F862ECE
:100E0C006530F2008930F3008231ED22853121000A
:100E1C0095178231E4228531AB30F2008830F30033
:100E2C008231ED228531210015082000BB003B08E2
:100E3C00C4004408BB00BC013B08AD003C08AE003C
:100E4C001030AF000030B000A03083312923853141
:100E5C00A030F2000030F30083310B238531823156
:100E6C00E4228531AF30F2008930F3008231ED227B
:100E7C00853124000C082000BB003B08C40044084A
:100E8C00BB00BC013B08AD003C08AE001030AF000D
:100E9C000030B000A030833129238531A030F2001E
:100EAC000030F30083310B2385318231E42285310C
:100EBC002000C101C201D92F9130F2008930F3001A
:100ECC008231ED22853120000C08BB003B08C400A8
:100EDC004408BB00BC013B08AD003C08AE00103020
:100EEC00AF000030B000A030833129238531A03011
:100EFC00F2000030F30083310B238531093083314C
:100F0C004C23853129302000BC009630BB007F304B
:100F1C00890B8E2FBB0B8E2FBC0B8E2F20000C1C25
:100F2C00982F992F9E2F313083314C238531A22F4E
:100F3C00303083314C23853120008C1CA62FA72FF9
:100F4C00AC2F313083314C238531B02F303083318D
:100F5C004C23853120000C1DB42FB52FBA2F313006
:100F6C0083314C238531BE2F303083314C23853176
:100F7C0020000C1EC22FC32FC82F313083314C23BD
:100F8C008531CC2F303083314C2385310D3083317A
:100F9C004C2385310A3083314C23853101302000BC
:100FAC00C1070030C23D003042020A300319410231
:100FBC00031CE12FE22F622FE22F803102283D30FB
:100FCC0084000030850008308231DE228731A03069
:100FDC0084000030850030308231DE2287312030B1
:100FEC0084000130850050308231DE2287312000B0
:100FFC008531742D013400340A34003464340034E7
:10100C00E8340334103427342034503472346F34C1
:10101C006A346534743420344D3450344C34413497
:10102C004234583420343A34203454344534533414
:10103C0054342034453454344134543420346434DE
:10104C0065347334203465346E34743472346534DE
:10105C006534733420344E346F346E34203443345E
:10106C006F346E346E346534633474346534653483
:10107C0073340D340A3400342034483461347234FF
:10108C006434773461347234653420343A34203427
:10109C0050344934433431343234463431343834B6
:1010AC0034343034203444344934503438342034DB
:1010BC002C34203446344F34533443342034693484
:1010CC006E347434653472346E34653420343D348B
:1010DC00333432344D3448347A3420340D340A34B9
:1010EC000034203443346F346D34703469346C34D0
:1010FC00653420346C346534203425347334203416
:10110C00613420342534733420345534543443340E
:10111C000D340A342034613476346534633420342D
:10112C00763465347234733469346F346E342034ED
:10113C0058344334383420343A3420342034253471
:10114C00643420340D340A3400346534743461341E
:10115C00743420344F345034543449344F344E3476
:10116C0020345234453447342034203461347634BE
:10117C0065346334203420346E3457345034553451
:10118C0045344E3420344D3453344234203462349C
:10119C0069347434203428343134323438342934BA
:1011AC0020343A3420340034203453346F347534C2
:1011BC007234633465343A34203431343234463446
:1011CC0031343834343430345F345434653473341B
:1011DC0074345F3465346E3474347234653465340D
:1011EC0073345F344E342E3443345F343234303401
:1011FC00323432342E3463340D340A340034203417
:10120C005434653473347434203473347534723418
:10121C0020346C34653473342034343420346934E1
:10122C006E34703475347434733420345234413425
:10123C0030342C345234413431342C345234413423
:10124C0032342C345234413434340D340A340034B6
:10125C002034553441345234543433342034333400
:10126C0038343434303430342034623464347334AD
:10127C00203454347834203473347534723420343C
:10128C0052344134353420340D340A340034203493
:10129C00563465347234733469346F346E3420349C
:1012AC003A342034333431342D34313432342D3417
:1012BC0032343034323432340D340A3400340D3498
:1012CC000A342034613476346534633420346E341B
:1012DC0057345034553445344E34203462346934E8
:1012EC0074343D3431340D340A34003420346134D8
:1012FC0076346534633420346E345734503455347A
:10130C0045344E3420346234693474343D343034D2
:10131C000D340A340034453474346134743420345C
:10132C00503469346E347334203450344F34523466
:10133C005434413420343A34003444346534633406
:10134C002034333431342034323430343234323487
:10135C00003465347434613474342034573450346C
:10136C005534413420343D340034313436343A343D
:10137C00313431343A3430343734003428346E3428
:0A138C0075346C346C3429340034DD
:020000040001F9
:08000000FF3FFF3FFF3FFF3F00
:04000E00C439FF3EB4
:00000001FF
